:1000000012C019C017C016C015C014C013C012C04A
:1000100011C010C00FC00EC00DC00CC00BC00AC074
:1000200009C008C007C011241FBECFE5D4E0DEBF61
:10003000CDBFC6C0E5CF1FB6EEE5F1E078E10CC05C
:1000400030E13A95F1F040B34470D9F70000000078
:10005000000000000000000024D0000040B30000B9
:10006000447041937A9539F035E13A9551F040B3B7
:100070004470D9F3E5CFEEE5F1E0909A9098768060
:100080001EC03FE0371B41F4EEE5F1E031963081D0
:10009000332309F00FC009C033941FBE30E43ABFC8
:1000A000189533E03A95F1F70895E4EFF0E078E140
:1000B00050D0F2CFEDE0F1E070E54BD0EDCFE6E7C8
:1000C000F1E0339631E030E13921319330E43921E8
:1000D000319330E43A21319330E83921319330E8DB
:1000E0003A213193319330E23A21319330E13A2190
:1000F000319330E23921319338E03921319334E0C2
:100100003921319331E03921319332E03921319372
:10011000E6E7F1E0882061F03FEF30A331A332A39E
:1001200033A334A335A336A337A33FEF30A309C0CD
:100130003FEF30A301A202A203A204A205A206A2DD
:1001400037A3772019F070E504D0A6CF70E401D072
:10015000A3CF31913323C9F400008A9A4FE04A9526
:10016000F1F700008A9842E04A95F1F77A9589F70D
:100170000000000000000000000000008A9A44E037
:100180004A95F1F700008A9808958A9A44E04A95C2
:10019000F1F7000000008A984CE04A95F1F7000062
:1001A00000007A95B1F60000000000000000000099
:1001B00000008A9A44E04A95F1F700008A98089571
:1001C00000240FEE05BB00E304BB0FEF08BB00E00B
:1001D00007BB0AEF02BB01E001BB02E005BF00E480
:1001E0000BBFB89AC098B998BA98C19AC29A000041
:1001F0000000000002E026B22094202249D0042D05
:10020000007111F002E0202EC5D08FD09AD0DBD043
:10021000882478943320F1F3222009F00EC04CD0CA
:10022000052D0073003369F5042D0272023249F581
:100230000FEF802E9924AA241DC02AD0052D007806
:100240000038F9F4042D027A023A29F40FEF802ED7
:100250009924AA2408C08824042D087A083A99F41D
:1002600000E39924A02E4DD013D04420E1F755206F
:10027000D1F707C046D020D04420A9F7552099F7E0
:1002800000C0882400C0942CA52C3BD03324C2CFBE
:100290001F9300E305BB31D030D000E205BB2DD069
:1002A00019D000E80223502E022F0074000F2F7384
:1002B000202B422E1F9108951F9300E305BB1DD0F4
:1002C0001CD000E205BB19D005D0422E03D0522E1F
:1002D0001F91089518E02227220F00E005BB03B309
:1002E00000950870069506950695202B06D000E22D
:1002F00005BB03D01A9581F708950EE10A95F1F731
:1003000008951F9317E60FEF0000000000000000A3
:100310000000000000000A95B9F70000000000008E
:1003200000001A9581F71F91089531E0E4EFF0E0A5
:1003300034963083339630833B96308336963083C1
:10034000089531E0EDE0F1E038963083389630835F
:100350003696319330833296319331933193308393
:10036000329630833296308337963083329631938B
:100370003193319331933193308335963083329674
:100380003193308335963083339631933083719631
:10039000308308954427E4EFF0E039E141933A9542
:1003A000E9F7EDE0F1E031E541933A95E9F7E6EB65
:1003B000F1E030E141933A95E9F7E6EBF1E00FEF38
:1003C000078307870895E6E7F1E0CDE0D1E000E498
:0E03D000499141930A95E1F741E04193089568
:1003DE00536E6573325769692076657273696F6EF5
:1003EE0020312E312C202843292032303037205214
:1003FE0061706861656C20417373656E6174203C39
:10040E007261706840726170686E65742E6E65748C
:10041E003E52656C656173656420756E646572200D
:10042E007468652047504C2E20536565206874749F
:10043E00703A2F2F7777772E726170686E65742EF3
:10044E006E65742F656C656374726F6E6971756518
:10045E002F78327769692F696E6465785F656E2EC5
:04046E007068700042
:00000001FF
